:0200000480007A
:100000006F004005732F2034930F8000630AFF03B5
:10001000930F90006306FF03930FB0006302FF038A
:10002000170F0000130F0F3363040F0067000F005A
:10003000732F203463540F006F00400093E19153FD
:10004000171F000023203FFC171F0000232E0FFA6C
:100050006FF01FFF930000001301000093010000E8
:10006000130200009302000013030000930300003A
:100070001304000093040000130500009305000022
:10008000130600009306000013070000930700000A
:1000900013080000930800001309000093090000F2
:1000A000130A0000930A0000130B0000930B0000DA
:1000B000130C0000930C0000130D0000930D0000C2
:1000C000130E0000930E0000130F0000930F0000AA
:1000D000732540F16310050097020000938202012E
:1000E000739052307350447497020000938202015F
:1000F00073905230735000189702000093820202EE
:1001000073905230B70200809382F2FF7390023BEB
:100110009302F0017390023A73504030970200004E
:1001200093824201739052307350203073503030BC
:100130009301000097020000938202ED7390523009
:10014000130510001315F501634C05000F00F00FA7
:10015000930110009308D005130500007300000000
:1001600093020000638A020073905210B7B200003D
:100170009382921073902230735000303725000024
:100180001305058073200530970200009382420119
:1001900073901234732540F173002030172400004F
:1001A000130444E6930440009301200097030000E9
:1001B0009383C3011303140003131400B7C3FFFF99
:1001C0009383C3BC631E7314930130009703000034
:1001D0009383C3011303140003531400B7C3000037
:1001E0009383C3BC631E7312930140009703000006
:1001F0009383C3011303140003231400B7C3AA9904
:100200009383C3BC631E73109301500097030000D7
:100210009383C3011303240003232400B7B39988F5
:100220009383B3AB631E730E9301600097030000CA
:100230009383C3011303340003233400B7A38877E7
:100240009383A39A631E730C93046000930160016F
:10025000970300009383030313031400A310040007
:1002600003030400630E030A03033400630A030A52
:10027000030314006316030A030324006312030A32
:100280009301700197030000938303031303540049
:10029000A32204000303440063040308030394003F
:1002A0006300030803035400631C03060303840074
:1002B00063180306930180019703000093830303EF
:1002C0001303A4002325040003039400630A03041A
:1002D0000303E400630603040303A400631203049E
:1002E0000303D400631E03029301900197030000EF
:1002F000938303031303F400A32704000303E40020
:100300006300030203033401630C03000303F400DE
:100310006318030003032401631403006310300215
:100320000F00F00F638001009391110093E1110021
:100330009308D00513850100730000000F00F00F33
:10034000930110009308D00513050000730000000E
:10035000F3222034E39692FCF322303463880200C7
:10036000E39062FC83820200E38C02FA7390133400
:0C03700073002030731000C0000000007B
:1010000000000000000000000000000000000000E0
:1010100000000000000000000000000000000000D0
:1010200000000000000000000000000000000000C0
:1010300000000000000000000000000000000000B0
:081040000000000000000000A8
:10200000DDCCBBAA998877665544332211EEFFEEEA
:1020100050505050505050505050505050505050C0
:1020200050505050505050505050505050505050B0
:1020300050505050505050505050505050505050A0
:102040005050505050505050505050505050505090
:102050005050505050505050505050505050505080
:102060005050505050505050505050505050505070
:102070005050505050505050505050505050505060
:102080005050505050505050505050505050505050
:102090005050505050505050505050505050505040
:1020A0005050505050505050505050505050505030
:1020B0005050505050505050505050505050505020
:1020C0005050505050505050505050505050505010
:1020D0005050505050505050505050505050505000
:1020E00050505050505050505050505050505050F0
:1020F00050505050505050505050505050505050E0
:10210000505050505050505050505050505050001F
:040000058000000077
:00000001FF
